:0200000480007A
:100000006F008004732F2034930F80006308FF0378
:10001000930F90006304FF03930FB0006300FF038E
:10002000130F000063040F0067000F00732F2034CC
:1000300063540F006F00400093E19153171F0000BD
:1000400023223FFC6FF09FFF732540F163100500F2
:10005000970200009382020173905230735000188F
:10006000970200009382020273905230B702008020
:100070009382F2FF7390023B9302F0017390023A75
:1000800097020000938282017390523073502030A7
:1000900073503030735040309301000097020000DD
:1000A000938282F673905230130510001315F501F8
:1000B000634C05000F00F00F930110009308D0056A
:1000C000130500007300000093020000638E02001D
:1000D00073905210B7B20000938292107390223046
:1000E00073232030E39A62F4735000303725000008
:1000F0007320053073503000970200009382420154
:1001000073901234732540F1730020309301200066
:1001100017250000130505EF8326050013052000B1
:10012000537005D073101000530500E0631AD50614
:100130009301300017250000130505ED8326050007
:100140001305E0FF537005D073101000530500E055
:100150006318D5049301400017250000130505EB33
:100160008326050013052000537015D0731010006E
:10017000530500E06316D5029301500017250000D7
:10018000130505E9832605001305E0FF537015D01C
:1001900073101000530500E06314D50063103002A3
:1001A0000F00F00F638001009391110093E11100A3
:1001B0009308D00513850100730000000F00F00FB5
:1001C000930110009308D005130500007300000090
:1001D000731000C0000000000000000000000000DC
:1001E000000000000000000000000000000000000F
:0C01F00000000000000000000000000003
:1010000000000000000000000000000000000000E0
:1010100000000000000000000000000000000000D0
:1010200000000000000000000000000000000000C0
:1010300000000000000000000000000000000000B0
:081040000000000000000000A8
:1020000000000040000000C0000000400000804FC1
:040000058000000077
:00000001FF
